:100000000C9462000C94C81A0C94F51A0C948A0093
:100010000C948A000C948A000C948A000C948A0038
:100020000C948A000C948A000C948A000C948A0028
:100030000C948A000C948F0B0C948A000C948A0008
:100040000C94221B0C948A000C949E1E0C94E11EAE
:100050000C948A000C948A000C948A000C948A00F8
:100060000C94F0080C948A000000000700020100C4
:100070000003040600000000000000000102040864
:100080001020408001020408102001020408102002
:10009000040404040404040402020202020203032E
:1000A00003030303000000002300260029000000D2
:1000B0000000250028002B0000000000240027007D
:1000C0002A00CF1F11241FBECFEFD8E0DEBFCDBF67
:1000D00012E0A0E0B1E0E2E1F2E402C005900D928E
:1000E000A23DB107D9F714E0A2EDB2E001C01D9224
:1000F000AC3BB107E1F710E0C4ECD0E004C02297BC
:10010000FE010E94E420C23CD107C9F70E940B20E7
:100110000C9407210C9400008091BE03813019F4E7
:1001200082E08093BE038091BE03833019F484E0A3
:100130008093BE030895A8950895CF93DF93FC01A3
:10014000962F9270862F817060FF20C0992331F026
:100150008091500380831092D20216C0A091D202E7
:10016000C091E903C770D0E0C656DD4F8881A8175B
:1001700010F080E03CC081E08A0F8093D202B0E0B2
:10018000A050BD4F8C91808381E031C09923C1F094
:1001900090819093D3021092D202292F207E203694
:1001A00051F490915003923020F390819F7190937D
:1001B000920393E01AC09E3F39F71092500317C084
:1001C0009091D3029F3F01F79091D202993288F625
:1001D00021E0290F2093D2023081E92FF0E0EF5384
:1001E000FC4F3083293281F691E090935003DF91E8
:1001F000CF910895DC01ED91FC910190F081E02D0B
:1002000009950895DC01ED91FC910190F081E02DBC
:10021000099508952091BF033091C003382748E025
:10022000C901880F991F37FF06C09C0151E225279D
:1002300050E1352701C09C01415091F73093C00334
:100240002093BF0308958436910520F4BC0180E01B
:1002500090E017C09C018E3B910528F42A55310986
:10026000AAE0B0E00CC0823D910528F4245B31097E
:10027000A4E6B0E004C02D5C3109A8E5B2E00E941C
:100280001820A4E6B0E09B01AC010E94272008954D
:1002900090E08C599F4F0E942301089582E0809343
:1002A000EA031092EB0391E09093EC038093ED034B
:1002B00083E08093EE0384E08093EF0385E08093F6
:1002C000F00384E28093F10385E28093F2030895C2
:1002D00060E08CE00E94301C61E08BE00E94301CEA
:1002E00061E08DE00E94301C60E082E00E94301CE2
:1002F00061E084E00E94301C089542E050E06CE828
:1003000070E080E00E94A81A0895E3E0F0E089E040
:1003100080935700E491E67081E0E63009F080E0D8
:100320000895CF93DF93C82F0E948501882381F021
:10033000DFB781E08093BD03F8940E949B0088E1C1
:1003400080936000C0936000C1110E949B00DFBFDA
:10035000DF91CF910895FC0140A5842F877090E034
:10036000959587950196242F217030E0820F931F79
:10037000880F880F08958F929F92AF92BF92CF926D
:10038000DF92EF92FF92CF93FC01C0A5EC2FE770B4
:10039000F0E0E656FD4FA081B0E0C7FF03C024E1C6
:1003A00030E002C02FE030E0FC0197A183E1989F8C
:1003B000F0011124E25AFE4F80809180A280B38028
:1003C000A20FB31F20E43FE14DE750E00E9432202E
:1003D000A50194010E946A208C2F887149F469015B
:1003E0007A01E0EDCE0EE7E0DE1EE11CF11C1BC041
:1003F000C7FF05C060E47AE88CE29EE004C060E0DC
:100400007EEE8AEB9BE069017A01F8EBCF0EFBE010
:10041000DF1EE11CF11CA50194010E946A20C20E9E
:10042000D31EE41EF51EC701B60169517C4F8F4FE4
:100430009F4F28EE33E040E050E00E946A20A8EE93
:10044000B3E00E942720CF91FF90EF90DF90CF90F4
:10045000BF90AF909F908F900895DB01FA01582FC5
:10046000569590E02481237030E0322F222740817E
:10047000240F311D11963C932E9344814C702181A1
:1004800030E060E4469F200D311D112413963C930B
:100490002E93129744814073228130E060E1469FA1
:1004A000200D311D112415963C932E9314974481F1
:1004B000407C238130E064E0469F200D311D1124F3
:1004C00017963C932E931697359618969F5F59175B
:1004D00048F680FF47C04081429546954695437057
:1004E0002DE431E0429FC001439F900D11240C96F2
:1004F00011969C938E93808190E074E096958795F9
:100500007A95E1F783709927829FA001839F500D10
:10051000929F500D1124445F5F4F13965C934E934E
:100520001297808190E09695879596958795837030
:100530009927829FA001839F500D929F500D1124F7
:10054000445F5F4F15965C934E93149740814370C0
:10055000429FC001439F900D11240C9617969C93C7
:100560008E9316970895803223E0920708F1883E13
:1005700023E0920740F48F519340E4E096958795ED
:10058000EA95E1F70895803D27E0920718F48C5D25
:1005900093400895883928E0920768F4885C974072
:1005A00074E0969587957A95E1F78D509C4F089564
:1005B00080E090E008958FEF93E008958C309105EE
:1005C00040F4A4E0880F991FAA95E1F7885D9C4F3D
:1005D0000895843F23E0920718F484529C4F0895B5
:1005E000811524E0920740F48657934FF4E0880F7A
:1005F000991FFA95E1F7089580E998E008959C0124
:100600003695279525753575821B930B9C012373B1
:100610003373969587959695879583739373820F19
:10062000931F9C0154E0369527955A95E1F7280FC2
:10063000391F2F703F7041E051E0249FC001259F7A
:10064000900D349F900D1124892F08952D988823A3
:1006500019F000002B9A02C000002B9800002D9A80
:10066000000008952D9A000083B12D980000829516
:1006700081700895CF93DF93D82F5C9A2D985C9862
:10068000C8E08D2F80780E942603DD0FC150C9F786
:100690002D98DF91CF9108958F770E943A030895A6
:1006A000CF93DF93D82FC8E08D2F80780E94260348
:1006B000DD0FC150C9F72D98DF91CF910895CF93E9
:1006C000DF932D98C8E080E0D82FDD0F0E94320321
:1006D0008D0FC150C9F7DF91CF9108950E944C034F
:1006E0000E945F035C9A0895A1E0B0E0EAE7F3E0BE
:1006F0000C94BB20806869830E943A036981862F2D
:100700000E9450035C9A2196E2E00C94D720CF938C
:10071000C091CA03C827E82FF0E0EF53FC4F67856C
:1007200089E70E9474036C2F8DE30E9474036C2F81
:1007300082E40E947403CF91089586E20E946E03C2
:100740000895CF938BE20E946E03C82F8CE20E9423
:100750006E03282F30E066E0369527956A95E1F71D
:1007600044E0C49FC0011124822B932BCF910895A4
:10077000CF93DF93EC016C818CE10E9474036D8157
:100780008DE10E9474036E818EE10E9474036F817B
:1007900080E20E947403688581E20E947403698587
:1007A00082E20E9474036A8583E20E9474036B856F
:1007B00084E20E9474036C8585E20E9474036D8557
:1007C0008AE20E9474036E858EE60E9474036F8530
:1007D0008FE60E947403688980E70E947403698928
:1007E00081E70E9474036A8982E70E947403DF91A3
:1007F000CF910895CF92DF92EF92FF92CF93DF9344
:100800006B017C01C11488E3D8068CE9E8068CE111
:10081000F80628F5C701B60120E836E948E950E0B6
:100820000E946A20E901689760E879E687E69FEF11
:100830000E943A206C0D7D1D8E1D9F1DF2E0660FFB
:10084000771F881F991FFA95D1F721E732E040E022
:1008500050E00E946A20F22EE32E80E421C0C701FE
:10086000B60120E03DE241E351E00E946A20E90147
:10087000689760E073ED8EEC9EEF0E943A206C0D5D
:100880007D1D8E1D9F1D660F771F881F991F21E7F5
:1008900032E040E050E00E946A20F22EE32E80E633
:1008A0006C2F6F71680F85E70E9474036E2D86E7C9
:1008B0000E9474036F2D87E70E947403DF91CF912C
:1008C000FF90EF90DF90CF9008958F929F92AF921C
:1008D000BF92CF92DF92EF92FF92CF93DF93D82F08
:1008E00083E00E946E038093BC0384E00E946E0349
:1008F0008093BB0360E086E00E94740361E087E0C0
:100900000E9474036FE789E00E94740365E08AE047
:100910000E94740362E18BE00E94740365E18CE045
:100920000E9474036DEF8DE00E94740360E08EE01E
:100930000E947403DD2319F08BE491E008C020913C
:10094000E80333E1239FC0011124825A9E4F0E9485
:10095000B8036CE880E30E9474036FE082E30E94B6
:10096000740362E483E30E9474038091E90387FFC8
:1009700002C064E101C06AE084E30E9474036AE299
:1009800085E30E9474036DE286E30E94740364EDC4
:1009900087E30E94740360E088E30E94740360E0D0
:1009A00089E30E947403D11109C0C090CA03D0909A
:1009B000CB03E090CC03F090CD0307C0C5E9CC2E6B
:1009C000C1ECDC2EED2CCEEDFC2ECAE38F2C99244D
:1009D000AA24BB24682D8C2F0E947403682D85E007
:1009E0008C0F0E947403FE2CED2CDC2CCC24CF5FEA
:1009F000CE3361F76FEF83E40E9474036FEF84E4FA
:100A00000E9474036FEF85E40E9474036FEF86E425
:100A10000E947403DD2311F066E002C06091CE03F2
:100A20008DE60E94740360E089E70E947403609180
:100A3000CF038AE70E94740360E083E70E94740397
:100A400060E084E70E947403D11109C06091C6037D
:100A50007091C7038091C8039091C90304C060E0FE
:100A600071EA8CEB93E30E94FA03DF91CF91FF9040
:100A7000EF90DF90CF90BF90AF909F908F900895B0
:100A800061E087E00E94740364E28EE70E947403D1
:100A900063E088E00E94740360E088E00E947403D1
:100AA00065E087E00E94740362E085E00E947403C1
:100AB00083E00E946E038093BC0384E00E946E0377
:100AC0008093BB03089583E00E946E038093BC0370
:100AD00084E00E946E038093BB0361E087E00E9484
:100AE00074036AE070E080E090E00E949B1B0E942B
:100AF000400500000895CF92DF92FF920F931F935D
:100B0000CF93DF931F92CDB7DEB7082F162F8EE35A
:100B100099830E947403F02EC02E9981D92E8C2DBA
:100B20008F19811738F4F60161916F018FE70E94E8
:100B30007403F5CF64E085E00E94740383E00E94B3
:100B40006E038093BC0384E00E946E038093BB031A
:100B50000E94781B6093B7037093B8038093B90326
:100B60009093BA0369E087E00E94740381E0809368
:100B7000BE030F90DF91CF911F910F91FF90DF90F7
:100B8000CF9008950F931F930E947B058091BE0321
:100B9000813099F40E94781B0091B7031091B8033B
:100BA0002091B9033091BA03601B710B820B930B38
:100BB000603A76488140910548F38091BE038130C8
:100BC00031F46EEB71E082E194E00E943A1D1F91D6
:100BD0000F9108950F931F938091BE03823021F4EB
:100BE0001092BE0381E020C08091BE038130D9F411
:100BF0000E94781B0091B7031091B8032091B903AC
:100C00003091BA03601B710B820B930B613A7648EB
:100C10008140910540F061E087E00E9474031092EA
:100C2000BE0382E001C080E01F910F910895EF9212
:100C3000FF920F931F93CF93DF938B019C01442767
:100C400037FD4095542F60E271EA87E090E00E9402
:100C50008C20E9011C161D0614F0C1E0D0E0D8017B
:100C600020E231EA47E050E00E9432209E01442712
:100C700037FD4095542F0E948C20790100E010E050
:100C80000E151F055CF42B9ACE010E94C11B2B98F8
:100C9000CE010E94C11B0F5F1F4FF2CFCDB7DEB751
:100CA000E6E00C94D320CF93DF935D9A6091FA0332
:100CB0007091FB038091FC039091FD030E94FA0365
:100CC00060E089E70E94740361E070E080E090E0FA
:100CD0000E949B1B0E949D03C82F61E070E080E092
:100CE00090E00E949B1B0E949D03D0E0C80FD11D85
:100CF00061E070E080E090E00E949B1B0E949D03F9
:100D0000C80FD11D61E070E080E090E00E949B1B65
:100D10000E949D035D989E01280F311DC901969583
:100D2000879596958795DF91CF910895CF93C82F9A
:100D30005D9A83E00E946E038093BC0384E00E946E
:100D40006E038093BB0360E086E00E94740361E061
:100D500087E00E9474036FE789E00E94740365E0F6
:100D60008AE00E94740362E18BE00E94740365E1F3
:100D70008CE00E9474036DEF8DE00E94740360E0CC
:100D80008EE00E9474036CE280E70E94740360E0CE
:100D900080E30E94740360E089E70E94740365E0C9
:100DA0008AE70E94740362E181E70E94740362E0B3
:100DB00082E70E94740360E083E70E94740360E0AE
:100DC00084E70E9474036091FA037091FB038091A1
:100DD000FC039091FD030E94FA0367E08DE60E94F8
:100DE00074036AE070E080E090E00E949B1B69E081
:100DF00087E00E9474036AE070E080E090E00E9467
:100E00009B1BCC2369F0C5E1C15009F459C061E0D6
:100E100070E088EB91E00E9417060E949B00F4CFDF
:100E200061E070E088E891E00E9417060E949B0054
:100E300065E08DE60E9474036AE070E080E090E077
:100E40000E949B1B61E070E088EB91E00E94170616
:100E50000E949B0064E08DE60E9474036AE070E0EB
:100E600080E090E00E949B1B61E070E08DE591E0E6
:100E70000E9417060E949B0062E08DE60E947403A8
:100E80006AE070E080E090E00E949B1B61E070E00F
:100E90008FEA90E00E9417060E949B0060E08DE6BA
:100EA0000E9474036AE070E080E090E00E949B1B67
:100EB00062E070E085E091E00E9417060E949B00CE
:100EC00061E087E00E9474035D98CF910895CF930D
:100ED000DF93EC014AE050E06D2F70E082E194E096
:100EE0000E94FF1D6EE282E194E00E941E1DBE0181
:100EF00084E0769567958A95E1F76F7077274AE0E9
:100F000050E082E194E00E94FF1D6EE282E194E0F5
:100F10000E941E1DBE016F7077274AE050E082E1FB
:100F200094E00E94FF1DDF91CF910895D82FC0E07B
:100F3000CD1780F45E9A64E670E080E090E00E9455
:100F40009B1B5E9864E670E080E090E00E949B1B33
:100F5000CF5FEECF6CE271E080E090E00E949B1BDF
:100F6000E6CF0F931F93CF93DF93EC01062F15E08D
:100F7000115051F0CE010E94F120081741F0602F6E
:100F8000CE010E94F920F4CF82E00E949607DF9103
:100F9000CF911F910F910895A0E0B0E0E2EDF7E04E
:100FA0000C94AD20482E562EC0E0D0E0612C712C60
:100FB000E12CF12C00E010E0442079F081E04816AB
:100FC000A1F092E0491219C028E4622E712C30E29F
:100FD000E32EF12C03E513E010C0612C712C6BE1C2
:100FE000E62EF12C0AEE13E008C04DE1642E712CC0
:100FF00059E2E52EF12C01EC13E043018C0E9D1E0D
:101000001092C0031092BF033401A62CA818B12C73
:10101000C30101966C01AE14BF04A8F4A00EB11E6A
:10102000511006C0C3010E94F120F501808305C064
:10103000F5016081C3010E94B107F50180810E9422
:101040000A013601E2CFC301511018C0C3010E944A
:10105000F120B82EC6010E94F1202B2D30E0322F56
:101060002227282B8091BF039091C00382179307FA
:1010700079F4C0E0D0E0552453949ECF36016091BE
:10108000C0030E94B1076091BF03C6010E94B1076F
:10109000D395C13093E0D90708F48ECF852DCDB715
:1010A000DEB7E0E10C94C92060E081E00E94CC074B
:1010B000882331F081E09091C103983309F080E0FA
:1010C000089561E081E00E94CC07089561E082E02C
:1010D0000E94CC07089560E082E00E94CC07811155
:1010E00008C0E3E5F3E01192119283E0E337F807DB
:1010F000D1F70895A1E0B0E0E0E8F8E00C94BB205F
:1011000089830E944E0192E09093F8039FEF9093A1
:10111000F9039AE0909302041092030410920404DD
:101120001092FA031092FB031092FC031092FD033D
:101130002EE12093FE039093FF0328EB3BE03093D6
:101140000104209300048981882371F061E080E02C
:101150000E94CC07E3E5F3E01192119283E0E337BC
:10116000F807D1F70E9466082196E2E00C94D72098
:1011700060E080E00E94CC07811103C081E00E9402
:101180007A080895CF93C1E0811101C0C0E06C2FAF
:1011900082E10E94691C6C2F83E10E94691C1092FD
:1011A000B1031092B0038091B9008C6F8093B900A5
:1011B00080E28093B80085E48093BC00CF910895CD
:1011C00085ED8093BC008091BC0084FDFCCF089528
:1011D000ECEBF0E0108285E480831092B003089578
:1011E0001F920F920FB60F9211242F933F934F939C
:1011F0005F936F937F938F939F93AF93BF93EF937F
:10120000FF93CF93DF931F92CDB7DEB78091B900E4
:10121000887F803609F4C7C0A8F5883209F464C015
:1012200098F4803109F45DC038F4882309F4F3C0E0
:10123000883009F456C0F1C0883109F455C08032B5
:1012400009F0EBC082E0A7C0803409F477C078F4DD
:10125000803309F45FC0883309F0DFC084E08093F5
:10126000AF038091B0038B7F8093B003D0C08035F3
:1012700009F452C0883509F467C0883409F0CDC03C
:1012800085E089C0883909F4C0C0A8F4883709F41A
:101290008AC038F4883609F486C0803709F483C0E0
:1012A000BCC0883809F4B1C0803909F47FC08038E7
:1012B00009F0B3C07BC0803B09F493C038F4803A96
:1012C00009F48CC0883A09F48CC0A7C0803C09F4AA
:1012D0009EC0883C09F49BC0883B09F09EC080E01A
:1012E00081C08091B40313C08091B1039FEF980F28
:1012F0009093B1038823D1F1E091B203F091B3034D
:10130000CF0101969093B3038093B20380818093C1
:10131000BB007DC083E03FC0E091B203F091B30316
:10132000CF0101969093B3038093B2038091BB00E9
:1013300080838091B10381508093B1038091B10388
:10134000823008F064C061C0E091B203F091B30351
:10135000CF0101969093B3038093B2038091BB00B9
:1013600080838091B10381508093B1038091B00359
:101370008B7F8093B0038091B00380FF4CC080913D
:10138000B0038E7F8093B0038091B003826080931E
:10139000B00384EA3DC08093AF038091B0038B7F9C
:1013A0008093B00338C01092B10331C0E091B5030F
:1013B000F091B603309749F18091BB008983809109
:1013C000B10391E0980F9093B103811102C062E0E4
:1013D00001C060E0CE010196099515C00E94E008A9
:1013E00016C081E0E091B503F091B603309769F043
:1013F000882311F063E001C061E0CE0101960995F8
:1014000099819093BB00811102C085E801C085ECF1
:101410008093BC0002C00E94E0080F90DF91CF9142
:10142000FF91EF91BF91AF919F918F917F916F91BC
:101430005F914F913F912F910F900FBE0F901F9092
:1014400018958F929F92AF92BF92CF92DF92EF92B8
:10145000FF92CF93DF93EC010E94781B6B017C011C
:101460004E01A12CB12C8091B00382FF11C02097B6
:10147000D1F30E94781B6C197D098E099F0986168D
:101480009706A806B90678F70E94E80881E004C02C
:101490008091AF031092AF03DF91CF91FF90EF9057
:1014A000DF90CF90BF90AF909F908F900895A2E073
:1014B000B0E0EDE5FAE00C94B720182F7B01022F85
:1014C000047022FD05C080910B0190910C0102C0B7
:1014D00080E090E02A8349830E94210A2A81498181
:1014E000811136C01092AF034093B103F092B30361
:1014F000E092B203110F1093B4039091B00321FF57
:1015000002C085E001C084E0892B8093B003809104
:10151000B00381FF0BC08091B0038D7F8093B00337
:101520008091B4038093BB0085EC01C085EE80936D
:10153000BC00822F817020FF0BC0011105C080917B
:101540000B0190910C0102C080E090E00E94210A02
:101550002296E6E00C94D320A2E0B0E0E2EBFAE0C1
:101560000C94B720182F7B01022F047022FD05C0B8
:1015700080910B0190910C0102C080E090E02A83E1
:1015800049830E94210A2A814981811138C0109221
:10159000AF034093B103F092B303E092B203812F03
:1015A000880F81608093B4039091B00321FF02C043
:1015B00085E001C084E0892B8093B0038091B00363
:1015C00081FF0BC08091B0038D7F8093B003809129
:1015D000B4038093BB0085EC01C085EE8093BC0012
:1015E000822F817020FF0BC0011105C080910B017B
:1015F00090910C0102C080E090E00E94210A2296A6
:10160000E6E00C94D320A0E0B0E0E9E0FBE00C942D
:10161000B5200E94781B0091AB031091AC03209180
:10162000AD033091AE036B017C01C01AD10AE20A0E
:10163000F30A9701860141E1C41647E2D406E104AA
:10164000F10408F442C02091AA0331E0320F309334
:10165000AA0320FF02C017E001C010E06093AB03B3
:101660007093AC038093AD039093AE0363E070E09E
:1016700082E194E00E94020161E070E082E194E086
:101680000E94020107E0010F812F90E0EC01CC0FD6
:10169000DD1FC35FDE4F68817981672F7727637015
:1016A0007727880F991F880F991F682B792B82E164
:1016B00094E00E94FA0068817981772782E194E0C2
:1016C0000E94FA001F5F1013DFCFCDB7DEB7E8E04E
:1016D0000C94D12025B190E0FC01EE0FFF1FE80F24
:1016E000F91FE65EFC4F8081282B25B988B19181D6
:1016F000892B88B98BB19281892B8BB9089585B1DB
:1017000090911703892385B988B190911803892393
:1017100088B98BB19091190389238BB908951F92D1
:101720000F920FB60F9211242F933F934F935F9315
:101730006F937F938F939F93AF93BF93CF93EF93C9
:10174000FF93C091760380910601C81708F03EC050
:1017500080911503909116039093870080938600E3
:10176000EC2FF0E0EE0FFF1FE35FFE4F80819181D1
:101770000E94DE02880F991F909316038093150331
:101780008091150390911603209107013091080173
:10179000281B390B30930801209307018091000426
:1017A00090910104880F991F2817390720F490930E
:1017B00008018093070180917403811142C08091D8
:1017C000F80380FF41C0C830E0F53EC080911503AA
:1017D0009091160390938700809386008091070173
:1017E00090910801909316038093150380917403E0
:1017F000882319F08FEF9FEF06C080911503909119
:10180000160388559240909389008093880080E465
:101810009CE9909308018093070180918400909146
:1018200085008097D0F30E947F0B80917503811112
:1018300005C08091060181500E946A0B10927603C8
:1018400027C08FEF9FEF06C080911503909116037C
:1018500088559240909389008093880080918400FD
:10186000909185008097D0F30E947F0B8091750343
:10187000811104C080917603811106C080917603A6
:101880008F5F8093760304C081500E946A0BF6CF6D
:10189000FF91EF91CF91BF91AF919F918F917F91E8
:1018A0006F915F914F913F912F910F900FBE0F90CD
:1018B0001F90189524E0829FC00111248C3091055F
:1018C00038F0853F23E0920728F084EF93E00895F5
:1018D0008CE090E00895CF93DF93C091F903C0337B
:1018E00090F48C2F807339F0803141F4809177032C
:1018F0008295807F05C080917C0302C080917D032A
:10190000CF70D0E015C0CF33E0F4CF70D0E080913D
:1019100077038295807F0E945A0CDE01AA0FBB1FBD
:10192000A35FBE4F11969C938E93219680917D0369
:101930000E945A0CFE01EE0FFF1FE35FFE4F9183E2
:101940008083DF91CF9108958091780390917903FE
:101950009F770E94FF02809377038F3029F4809154
:101960007D038695805804C099E0899F802D1124BD
:1019700080937C03F8940E946B0C78948091ED0323
:101980008132E1F480917C039FEF980F9E3F78F0C5
:101990008091B0008F7D8093B00061E080917C03E6
:1019A000811101C060E083E00E94691C089580936A
:1019B000B4008091B00080628093B0000895FF92DF
:1019C0000F931F93CF93DF930BEE13E0C0E0D0E0B3
:1019D000B3E0FB2E8C2FD801ED918D019E2F907FCF
:1019E0009031F1F4EF70F0E0EE0FFF1FE35FFE4F78
:1019F000208131816F2D0E944A20E92FF0E0EE0F07
:101A0000FF1FEC56FD4F61E08081918182179307A3
:101A100008F060E0FE01EE55FD4F80810E94691CD8
:101A20002196C830D105B1F6CDB7DEB7E5E00C940C
:101A3000D4200F931F93CF93DF9303E513E0C0E00F
:101A4000D0E02091F903822F8F7090E0C817D9075A
:101A5000E9F00196C817D90711F42033B8F4F8015A
:101A6000808191819F70892B79F0F894F8018081B1
:101A700091819F700E94B302FE01EE0FFF1FE35F92
:101A8000FE4F9183808378940E94DF0C21960E5F35
:101A90001F4FC031D105A9F6DF91CF911F910F9152
:101AA0000895FF920F931F93CF93DF9381EC93E000
:101AB0000E94AB01809306019091F903292F2F70AA
:101AC000281304C081E0820F8093060190539F3059
:101AD00060F44091060130E0842F90E001972817D0
:101AE000390719F44F5F4093060180910601813157
:101AF00018F080E180930601ECE1F3E0DF0112973A
:101B00001C92DF0111971C921082339683E0E4331C
:101B1000F807A1F74FEF3FEFACEAB2E00BEE13E0AE
:101B20002FEFE80189918E018031F8F490E0FD01FA
:101B300032976081FC01EE0FFF1FE80FF91FE65E90
:101B4000FC4F8081862B8083CD010197EC01588169
:101B50008181852B81839C918281892B82836095F1
:101B6000509590952923352346231396D3E0033FC0
:101B70001D07B9F6409317033093180320931903F8
:101B8000C2EAD2E00BEE13E0F12CF80181918F0153
:101B9000823230F08632B8F0863211F460E010C044
:101BA000F6E0FF1204C08091C1008F7E06C087E07E
:101BB000F81205C08091C100877F8093C10061E069
:101BC00088810E94301CF3942196E8E0FE12DDCF5C
:101BD0008091EB03803231F461E089E00E94691C5E
:101BE00082E801C082E08093800081E080937503E9
:101BF000809374038091ED03813211F08732D9F420
:101C000061E083E00E94301C60E083E00E94691C78
:101C10008091ED03813231F481E08093B0008093B4
:101C2000B10009C082E08093B00085E08093B100EC
:101C30008EE38093B3008AE1809381008FEF9FEF62
:101C4000909389008093880080ED97E090938700BF
:101C50008093860080E49CE99093080180930701BB
:101C600090931603809315031092760380916F0072
:101C7000816080936F008091F80383FF0DC0809195
:101C80005303909154039F70892B31F00E94190DDA
:101C90001092740310927503CDB7DEB7E5E00C9493
:101CA000D420CF93C82F8091F0038B3221F46C2F76
:101CB0008FE00E94691C8091ED03873249F4809186
:101CC000B000CC2311F0806101C08F7E8093B00002
:101CD000CF910895A4E2B0E0E0E7FEE00C94AB20E1
:101CE0006B017C010E946C1B4B015C0181E00E9436
:101CF000650483E08093BE030E9463056AEC71E093
:101D000082E194E00E943A1D7BE1272EE0E53E2E21
:101D1000F7E47F2EA6E44A2EB5E55B2EC114D1046C
:101D2000E104F10469F00E946C1B681979098A09C1
:101D30009B096C157D058E059F0510F080E0D5C0D0
:101D40008091BE03843051F768ED71E082E194E048
:101D50000E943A1D8FE70E944C030E945F038CA3F0
:101D6000823601F501EC13E00E945F03D8018D93E8
:101D70008D01B3E00A3E1B07B9F78091C103883398
:101D800009F0ADC061EE71E082E194E00E943A1D7D
:101D900082E48CA361E0CE0184960E94C2055D9A24
:101DA00081E0A3C0803741F0893611F581E00E94BF
:101DB0007A0889E4898304C03982C12CD12C760148
:101DC0009091BD038091F803992311F0806801C0C0
:101DD0008F778093F803EAEEF3E0DE011296822D0E
:101DE00001900D928A95E1F76CE1CE01019675C0E4
:101DF0008437E1F4E4E5E98383E08A8384E88B8334
:101E000088E08C838FE08D838EE1EDE2F1E0DE01EE
:101E1000169601900D928A95E1F763E2CE01019644
:101E20000E94C205C12CD12C760159C0853789F496
:101E30000AEE13E00E945F03D8018D938D01B4E098
:101E400005301B07B9F761E080E00E94CC075CA277
:101E500041C08636B9F44982E3E5F3E0AE014D5F57
:101E60005F4F208131813296CA010197DC013C939A
:101E7000DA012C934E5F5F4FB3E0E337FB0789F73E
:101E800061E2B3CF8736C9F403E513E00E945F0334
:101E9000682E0E945F03262D30E0322F2227280F64
:101EA000311DF801219331938F01F3E003371F07B0
:101EB00069F77CA20E9466080DC0873481F4E3E5CF
:101EC000F3E01192119283E0E337F807D1F70E9413
:101ED00066087CA261E0CE0184960E94C20583E080
:101EE0008093BE030E94400519CFA496E2E10C94B2
:101EF000C7201F93CF93DF93C82FD62F61E00E9496
:101F0000301C61E08C2F0E94691C61E08D2F0E94C3
:101F1000691C8AE090E00E94C11B8D2F0E949C1CCE
:101F2000892B71F060E08C2F0E94691C8AE090E0A0
:101F30000E94C11B8D2F0E949C1C11E0892B09F06F
:101F400010E060E08C2F0E94301C60E08C2F0E941B
:101F5000691C60E08D2F0E94691C812FDF91CF9159
:101F60001F91089580E48093BA001092BD008DE91E
:101F700090E09093B6038093B5031092500315E060
:101F800004E0C2E0FC2E80915003813039F480E0FF
:101F90000E946504F09250035E98F5CFC091500303
:101FA000C33061F45D98809192030E948703C093CF
:101FB000BE030E94400500935003E5CF809150037B
:101FC000843009F78091BE038430E9F68FE70E94E0
:101FD0004C03C0E0D3E0E091E903E770F0E0E6569F
:101FE000FD4F808190E09E01205033402817390733
:101FF00024F40E945F038993EECF109350035D9AFF
:10200000C2CFAAE2B0E0E7E0F0E10C94BA201FEF03
:10201000198389E2E1ECF3E0DE01129601900D9262
:102020008A95E1F721E04AE2BE016F5F7F4F80E2CF
:102030000E94570A81110EC021E041E0BE016F5F8E
:102040007F4F80E20E94AC0A811104C082E080933D
:10205000500302C01093500380915003823051F01E
:102060000E946C1B60934C0370934D0380934E034E
:1020700090934F03AA96E3E00C94D620A1E0B0E041
:10208000E4E4F0E10C94BB20809150038230D9F459
:1020900080919203805A898321E041E0BE016F5F05
:1020A0007F4F80E20E94570A882369F08FEF809368
:1020B00050030E946C1B60934C0370934D038093FC
:1020C0004E0390934F032196E2E00C94D720A1E0B9
:1020D000B0E0EDE6F0E10C94BB208091500382303B
:1020E000D1F421E041E0BE016F5F7F4F80E20E94AA
:1020F000AC0A882371F08FEF809350030E946C1B11
:1021000060934C0370934D0380934E0390934F0361
:1021100002C0898101C08FEF2196E2E00C94D720A4
:10212000A2E2B0E0E6E9F0E10C94AB209E012F5F63
:102130003F4F80E1D9011D928A95E9F76CEE71E07D
:1021400082E194E029A33AA30E943A1D0E9463050C
:102150001D8A1E8A1F8A188E312C212C00E0812CAA
:10216000912C5401412C84E7582E8BE8682E82E391
:10217000782E90E5C92E93ECD92EE12CF12C84EF2A
:1021800091E0A0E0B0E08D8F9E8FAF8FB8A380E08C
:102190009EECADEEB4E3898F9A8FAB8FBC8F80E05D
:1021A00094E7ABE8B2E3898B9A8BAB8BBC8B82E173
:1021B00094E00E94061E892B09F4E1C082E194E0BC
:1021C0000E94331E9C0133272C32310509F442C092
:1021D000ACF42332310509F0ABC019821A821B829C
:1021E0001C821D821E821F82188619861A861B86F3
:1021F0001C861D861E861F86188A60C02434310501
:1022000029F02335310509F4B2C092C064E482E1BB
:1022100094E00E941E1D2AE030E040E054E76BE8A5
:1022200072E382E194E00E949A1D6CE282E194E004
:102230000E941E1D2AE030E040E05EEC6DEE74E38B
:1022400082E194E00E949A1D6CE282E194E00E9497
:102250004C1DADCF0F5F043009F0A9CF29813A8121
:102260004B815C81A8EEB3E00E942720698B7A8BBA
:102270008B8B9C8B2D813E814F8158850E9427201E
:10228000698F7A8F8B8F9C8F29853A854B855C85EA
:102290002D8F3E8F4F8F58A32D853E854F855889B2
:1022A0000E9427206B017C0160323EE473078105A8
:1022B000910530F462E38CE10E94740300E077CF73
:1022C000603345E774078105910510F462E2F3CFAE
:1022D00060345CE975078105910510F466E2EBCF87
:1022E00080E5C81683ECD806E104F10410F462E13D
:1022F000E2CF90E6C9169AEED906E104F10410F493
:1023000065E1D9CFA0E7CA16A1E1DA06A1E0EA06A5
:10231000F10410F461E0CFCFB0EACB16B6E8DB06EB
:10232000B1E0EB06F10410F463E0C5CF65E0C3CF84
:1023300010ED180F1A3008F03ACFE1E0F0E0EC0FA2
:10234000FD1F24E0029FE00DF11D11242081318149
:1023500042815381AAE0B0E00E942720610F711DE5
:10236000811D911D608371838283938320CF49886F
:102370005A886B887C88812C912C540118CF811449
:102380009104A104B10489F4C301B2010E94FA03CB
:1023900061E070E080E090E00E949B1B1D8A1E8A35
:1023A0001F8A188E312C22242A948D8D9E8DAF8DFC
:1023B000B8A188169906AA06BB06D0F40E949D0310
:1023C0002D893E894F89588D280F311D411D511D82
:1023D0002D8B3E8B4F8B588F381608F4382E821574
:1023E00008F4282E3FEF831A930AA30AB30A56C0B3
:1023F000C301B20128EE33E040E050E00E946A20C1
:10240000BA01A9012AE030E082E194E00E94E81DCF
:102410006CE282E194E00E941E1D4AE050E0632DD0
:1024200082E194E00E94F71D6CE282E194E00E9458
:102430001E1D6D897E898F89988DA50194010E944A
:102440006A20BA01A9012AE030E082E194E00E940A
:10245000E81D6CE282E194E00E941E1D4AE050E01B
:10246000622D82E194E00E94F71D6CE282E194E02B
:102470000E944C1D4C0C5D1C6E1C7F1C898D9A8D1E
:10248000AB8DBC8D84159505A605B70520F449884C
:102490005A886B887C88812C912C540129893A892F
:1024A0004B895C89283E33404105510509F07FCEB8
:1024B000A296E2E10C94C720A1E0B0E0E2E6F2E1EE
:1024C0000C94BB2080E00E94910161E085E00E94B5
:1024D000301C61E086E00E94301C0E94680160E0D0
:1024E00080E00E94301C61E081E00E94301C40E0EE
:1024F00052EC61E070E082E194E00E944E1F0E9485
:10250000B8080E946B0869EF71E082E194E00E94D4
:102510001B1D84E893E00E94670760E172E082E19E
:1025200094E00E941B1D4AE050E065E070E082E10B
:1025300094E00E94D01D0E947D0178945E9A63E130
:1025400083E00E94790F882329F05E985D980E94AD
:102550009010FBCF62E189E00E94790F811104C0E5
:102560000E945408811119C063E572E082E194E091
:102570000E941B1D60E070E0CB010E946A0E882360
:1025800049F00E94610868E172E082E194E00E94F3
:102590003A1D5D9A0E94510D10C00E94510D80910C
:1025A000EC03823209F0CAC08091EE03833209F055
:1025B000C5C08091F80381FDC7C08091EC038232D1
:1025C00031F58091EE03833211F581E00E94C2085B
:1025D0008091F80382FF08C063E372E082E194E037
:1025E0000E943A1D0E94B20F64E170E080E090E02A
:1025F0000E949B1B21E041E0BE016F5F7F4F80E2A4
:102600000E94AC0A811103C081E0809350036EE305
:1026100072E082E194E00E941B1D8FE00E94910114
:1026200080E00E9465041092920380E00E9487037C
:1026300080E0883170F08093D40283E08093BE0301
:102640000E94630580915003882371F00E9401105D
:102650000BC021E0280FE82FF0E0EF53FC4F9785E7
:10266000992349F3822FE5CF8091F203982F9D7F24
:10267000983229F440E052EC61E070E027C08932E2
:1026800071F440EA56E861E070E082E194E00E9473
:102690004E1F8091C20080628093C2001BC0809157
:1026A000E9038871803129F440E855E260E070E088
:1026B0000DC04091C2035091C3036091C403709157
:1026C000C5034A3051056105710570F382E194E05C
:1026D0000E944E1F82E194E00E94061E892B29F081
:1026E00082E194E00E94331EF5CF8091F1038432A1
:1026F00029F08091C1008F7E8093C1008091F20308
:10270000853241F08852833028F08091C100877F64
:102710008093C1001092D6021092D50210925203FB
:102720000E94781B60938E0370938F0380939003B5
:10273000909391032196E2E00C94D7208091F803C6
:102740008B7F8093F80335CF82FD37CF64EF71E044
:1027500080E090E00E946A0E882309F42ECF0E9448
:10276000610868E172E082E194E00E943A1D0E94F3
:10277000510D5D9A22CFCF93DF9382E194E00E94C6
:10278000061E892BE9F0C091D502D0E0CE0101965A
:102790008F7199272091D60230E08217930781F03C
:1027A00082E194E00E94331EC952DD4F88838091FC
:1027B000D50290E001968F7199278093D502DDCFE5
:1027C000DF91CF910895A0E0B0E0E9EEF3E10C9441
:1027D000B520D82FC62F0E94781B0091AB03109113
:1027E000AC032091AD033091AE036B017C01C01AA4
:1027F000D10AE20AF30A9701860141E1C41647E2D1
:10280000D406E104F10408F4D1C16093AB037093E2
:10281000AC038093AD039093AE0380910D01909132
:102820000E01880F991F80939303892F8770209141
:102830009403287F282B2093940380910F0190917B
:102840001001880F991F382F330F330F330F277064
:10285000232B20939403282F22952695277080916F
:102860009503807C9770990F990F990F822B892B74
:10287000809395032091110130911201220F331F93
:10288000922F9295990F990F907C8F73892B80933B
:102890009503932F9295990F990F907C822F86958F
:1028A0008695892B8093960332FB882780F92091A7
:1028B00097032E7F282B20939703809113019091EB
:1028C0001401880F991F382F330F2170232B209369
:1028D0009703382F331F3327331F20919803207F0E
:1028E000892F8770880F232B282B209398038091A2
:1028F000150190911601880F991F382F3295307F5E
:102900002F70232B20939803382F32953F702091FE
:1029100099032078892F87708295807F232B282B1D
:10292000209399038091170190911801880F991FA6
:102930002F7720939903292F27952227279586956E
:10294000822B80939A03892F8695837020919B0315
:102950002C7F282B20939B038091190190911A01C1
:10296000880F991F382F330F330F2370232B209399
:102970009B03382F329536953695337020919C0302
:10298000207E892F8770880F880F232B282B209378
:102990009C0380911B0190911C01880F991F382F77
:1029A0003295330F307E2F71232B20939C03929509
:1029B000990F907E869586958695892B80939D03A9
:1029C00080911D0190911E01880F991F80939E0395
:1029D000892F877020919F03287F282B20939F03A6
:1029E00080911F0190912001880F991F382F330F7C
:1029F000330F330F2770232B20939F03282F22950B
:102A0000269527708091A003807C9770990F990F6D
:102A1000990F822B892B8093A00320912101309163
:102A20002201220F331F922F9295990F990F907CBC
:102A30008F73892B8093A003932F9295990F990FF1
:102A4000907C822F86958695892B8093A10332FBFB
:102A5000882780F92091A2032E7F282B2093A203A0
:102A60008091230190912401880F991F382F330FF3
:102A70002170232B2093A203382F331F3327331FBA
:102A80002091A303207F892F8770880F232B282B69
:102A90002093A3038091250190912601880F991F0F
:102AA000382F3295307F2F70232B2093A303382F9C
:102AB00032953F702091A4032078892F87708295EA
:102AC000807F232B282B2093A403809127019091B2
:102AD0002801880F991F2F772093A403292F27956A
:102AE000222727958695822B8093A5039695937030
:102AF0008091A6038C7F892B8093A60320912901C6
:102B000030912A01220F331F922F990F990F837052
:102B1000892B8093A6032295269526952370809174
:102B2000A703807E932F9770990F990F822B892B83
:102B30008093A70320912B0130912C01220F331F8A
:102B4000922F9295990F907E8F71892B8093A70376
:102B5000832F8295880F807E269526952695282B93
:102B60002093A803DD2311F088E001C080E0CC238E
:102B700011F094E001C090E0892B8093A9036FE0ED
:102B800070E082E194E00E940201C3E9D3E0699120
:102B900082E194E00E94601E83E0CA3AD807B9F748
:102BA00060E070E082E194E00E940201CDB7DEB700
:102BB000E8E00C94D120CF93C82F682F82E194E0F5
:102BC0000E94601E8C2F0E940A01CF910895A0E000
:102BD000B0E0EDEEF5E10C94B520C82F0E94781B13
:102BE0000091AB031091AC032091AD033091AE0383
:102BF0006B017C01C01AD10AE20AF30A970186012F
:102C000041E1C41647E2D406E104F10408F445C0EA
:102C10006093AB037093AC038093AD039093AE03CA
:102C20001092C0031092BF0388EA0E94DB15CC23E8
:102C300011F081E801C081E00E94DB1580E10E9473
:102C4000DB1500E010E0F801EE0FFF1FE35FFE4F21
:102C5000808191810E94DE02EC01B3E0CC0FDD1F88
:102C6000BA95E1F78D2F0E94DB158C2F0E94DB15A2
:102C70000F5F1F4F0031110531F76091C00370E005
:102C800082E194E00E94FA006091BF037091C0035A
:102C9000772782E194E00E94FA00CDB7DEB7E8E042
:102CA0000C94D120AAE1B0E0E8E5F6E10C94AD2067
:102CB0000E949B008CE00E946E0381110BC06CE8A7
:102CC00072E082E194E00E943A1D80E00E94650477
:102CD0000E9463050E94BB130E94781B0E9467102C
:102CE00091E0853009F090E01FEF8091BE038430C1
:102CF00009F4FEC19111FCC17CC00E94A103909314
:102D00007B0380937A035D9AC0928E03D0928F03E7
:102D1000E0929003F0929103109251038091780316
:102D200090917903880F991F816090937903809324
:102D300078035E9880E00E94510E80910003982FE6
:102D40009E7309F02CC2F8948091E90341E053E0AE
:102D50006DE071E087700E942D020E946B0C7894E8
:102D60009091000380914A0390FF13C2811124C007
:102D700093E5E92E93E0F92E00E010E0F701808161
:102D8000918194FD0CC0F801EE0FFF1FE35FFE4F31
:102D9000808191810E94DE02D7018D939C930F5F09
:102DA0001F4FB2E0EB0EF11C0031110539F70E9404
:102DB000660881E080934A0380915203811103C029
:102DC00081E0809352031092730310927503109266
:102DD00074038091E903887109F009C20E94DF0C35
:102DE00083E08093BE030E94400581E080934B0303
:102DF0005D980E94781B4B015C010E946C1B6B016B
:102E00007C0180915103823008F063C040908E03B2
:102E100050908F03609090037090910380918A038B
:102E200090918B03A0918C03B0918D03841595052F
:102E3000A605B70509F44DC081EC93E00E94BB01E3
:102E40006C5D75408109910995018401041915098A
:102E5000260937096017710782079307D0F540925A
:102E60008A0350928B0360928C0370928D030E94B0
:102E70009D03282F80937E0380917F039091800390
:102E8000820F911D9093800380937F036091810353
:102E90006F5F609381036930E0F070E00E9456201C
:102EA0007093800360937F0380917D03E3E08E9FA6
:102EB000600D711D112476956795769567956093E1
:102EC0007D030E94A40C1092800310927F03109245
:102ED0008103809152030091D402882351F1109113
:102EE0005103101708F035C240908E0350908F03A5
:102EF0006090900370909103A50194012419350905
:102F0000460957092F8B388F498F5A8F81EC93E0F0
:102F10000E94BB0168517C4F8F4F9F4F2F89388D86
:102F2000498D5A8D621773078407950708F4D8C135
:102F300010C280918E0390918F03A0919003B09165
:102F4000910375016401C81AD90AEA0AFB0A81ECE7
:102F500093E00E94BB019B01AC01A02FB0E00E9456
:102F600027206C157D058E059F0558F480928E03F1
:102F700090928F03A0929003B092910381E080938E
:102F80004B0380917403811116C08091F203883243
:102F900019F40E94030B0FC0893239F46091510378
:102FA000809173030E94E31306C08A3221F480915A
:102FB00073030E94E71580914B03882309F472C0C4
:102FC000E0919203EF5FE0939203E83131F0F0E09B
:102FD000EF53FC4F8785811102C0109292038091BC
:102FE000FA039091FB03A091FC03B091FD03892BA0
:102FF0008A2B8B2B09F44EC080918203909183031E
:10300000A0918403B0918503892B8A2B8B2B09F423
:1030100041C00E945306082F10E020910901309111
:103020000A0136952795369527952C5E3F4F201738
:10303000310770F40E946C1B68517C4F8F4F9F4F7B
:10304000609382037093830380938403909385033A
:10305000C801880F991F880F991F4091090150914D
:103060000A019A01220F331F240F351F820F931F6D
:10307000969587959695879590930A018093090177
:103080006091C6037091C7038091C8039091C903F2
:103090000E94FA03809192030E9487030E943E10CF
:1030A00010924B03809150038F3F09F04DC20E9454
:1030B0006C1B00914C0310914D0320914E033091F5
:1030C0004F03601B710B820B930B693E73408105AC
:1030D000910508F439C20E946C1B60934C037093F5
:1030E0004D0380934E0390934F030E9401102CC216
:1030F0000E94781B6B017C018091BE038430D1F467
:103100008FE70E944C0300E013E0E091E903E770D1
:10311000F0E0E656FD4F808190E09801205033406A
:10312000281739070CF0E9CD0E945F03D8018D9371
:103130008D01EBCFE091E903E770F0E0E656FD4F3B
:1031400040814F5F21E0BE016F5F7F4F80E20E94B0
:10315000AC0A882371F0109350030E946C1B60939B
:103160004C0370934D0380934E0390934F0390E074
:10317000BCCDE091E903E770F0E0E656FD4F4081F9
:1031800050E0BE016E5F7F4F80E093E00E94E82038
:10319000BBCD882309F410CE10924A030DCE982F90
:1031A0009873983309F008CE9091F702892787FF2A
:1031B00003CE90589093F7028091F203853209F084
:1031C000FBCD10E0212F30E080910003877090E06C
:1031D000821793070CF4F0CD1F5FE12FF0E0E05071
:1031E000FD4F608182E194E00E94601EEBCF8091F0
:1031F000F70290910003982796FD66C0807C90E4CA
:1032000089278093F7028091D6023091D5028317E7
:10321000D1F0E8EFF2E020E02F5F90E0DC01A9526E
:10322000BD4F4C91419301968F719927283011F031
:103230008313F2CF8093D602295C8091F702282B6A
:103240002093F70241C080917E038093F802809121
:10325000EC03863211F482E105C08091EF038632DF
:1032600051F48EE00E94C51C95958795959587959C
:103270008093F90202C01092F9028091EE03863227
:1032800011F483E105C08091F003863251F48FE0A0
:103290000E94C51C95958795959587958093FA0210
:1032A00002C01092FA0280917A0390917B0390936E
:1032B000FB028093FC0280917803909179039F77C1
:1032C0000E94FF028093FD0269E087EF92E00E9476
:1032D0007B050E94EA05811181CD0E94BB13F9CFC5
:1032E0008091780390917903880F991F90937903C7
:1032F0008093780381E080934B03111110C0C0923A
:103300008603D0928703E0928803F092890310929B
:1033100082031092830310928403109285031F5F2F
:103320001093510381EC93E00E94BB01640D751D65
:10333000861D971D60938E0370938F038093900377
:10334000909391035E9A81E00E94510E0E94A40C1A
:1033500003C0101709F4A7C080915103882309F412
:1033600010CE809102048823D9F0909173039111BB
:1033700017C0409186035091870360918803709134
:10338000890346015701841A950AA60AB70A90E0F4
:103390000E942301681579058A059B0508F4B5C0CC
:1033A000809104048823D9F090917503911117C07E
:1033B000409186035091870360918803709189033F
:1033C00046015701841A950AA60AB70A90E00E949E
:1033D0002301681579058A059B0508F4ADC0809125
:1033E00003048823D9F090917403911117C0409180
:1033F0008603509187036091880370918903460189
:103400005701841A950AA60AB70A90E00E94230180
:10341000681579058A059B0508F492C08091FA0326
:103420009091FB03A091FC03B091FD03892B8A2BA3
:103430008B2B09F4A6CD8091820390918303A091F8
:103440008403B09185030097A105B10509F499CDD6
:10345000C81AD90AEA0AFB0AF7FC93CD8091F8034F
:10346000829581700E94960680E00E9465040E9409
:1034700040050E946C1B6B017C012091FF0330E032
:10348000A8EEB3E00E941820C60ED71EE81EF91E53
:103490006894C0F8C0928203D0928303E0928403C0
:1034A000F09285036ECD80918E0390918F03A09151
:1034B0009003B091910324013501481A590A6A0A10
:1034C0007B0A81EC93E00E94BB019B01AC01A12F20
:1034D000B0E00E942720641575058605970508F061
:1034E0003BCF109279031092780381E080934B03D5
:1034F00010927D030E94A40C80928E0390928F0301
:10350000A0929003B092910327CF81E08093730340
:103510000E94190D8091FE030E9448016C0D7D1DD3
:103520008E1D9F1D6160609382037093830380935F
:1035300084039093850334CF81E0809375034FCF4C
:1035400081E0809374036ACF6A96E0E10C94C9200D
:103550008230E8F4E82FF0E0EE0FFF1FEB5FFB4F47
:1035600071836083813041F0809169008C7F842B6E
:1035700080936900E89A089580916900440F551F6F
:10358000440F551F837F842B80936900E99A089527
:103590001F920F920FB60F9211242F933F934F93C8
:1035A0005F936F937F938F939F93AF93BF93EF93AB
:1035B000FF938091050490910604892B29F0E091F6
:1035C0000504F09106040995FF91EF91BF91AF9129
:1035D0009F918F917F916F915F914F913F912F912B
:1035E0000F900FBE0F901F9018951F920F920FB65D
:1035F0000F9211242F933F934F935F936F937F9379
:103600008F939F93AF93BF93EF93FF9380910704A2
:1036100090910804892B29F0E0910704F0910804A7
:103620000995FF91EF91BF91AF919F918F917F91FC
:103630006F915F914F913F912F910F900FBE0F901F
:103640001F9018951F920F920FB60F9211242F936F
:103650003F938F939F93AF93BF9380910A04909170
:103660000B04A0910C04B0910D043091090423E0E7
:10367000230F2D3720F40196A11DB11D05C026E8AA
:10368000230F0296A11DB11D2093090480930A0403
:1036900090930B04A0930C04B0930D0480910E043E
:1036A00090910F04A0911004B09111040196A11DF6
:1036B000B11D80930E0490930F04A0931004B09357
:1036C0001104BF91AF919F918F913F912F910F90D6
:1036D0000FBE0F901F9018952FB7F89460910A04B1
:1036E00070910B0480910C0490910D042FBF0895EC
:1036F0003FB7F89480910E0490910F04A0911004AC
:10370000B091110426B5A89B05C02F3F19F0019672
:10371000A11DB11D3FBF6627782F892F9A2F620FF9
:10372000711D811D911D42E0660F771F881F991F33
:103730004A95D1F70895CF92DF92EF92FF92CF93FF
:10374000DF936B017C010E94781BEB01C114D10453
:10375000E104F10479F00E94781B6C1B7D0B683E3C
:103760007340A0F381E0C81AD108E108F108C851FC
:10377000DC4FECCFDF91CF91FF90EF90DF90CF90B7
:1037800008950197009739F0880F991F880F991FA6
:1037900002970197F1F70895789484B5826084BD0B
:1037A00084B5816084BD85B5826085BD85B5816045
:1037B00085BDEEE6F0E0808181608083E1E8F0E0A5
:1037C0001082808182608083808181608083E0E8D4
:1037D000F0E0808181608083E1EBF0E080818460B3
:1037E0008083E0EBF0E0808181608083EAE7F0E0B5
:1037F0008081846080838081826080838081816019
:1038000080838081806880831092C1000895833016
:1038100081F028F4813099F08230A1F0089586304B
:10382000A9F08730B9F08430D1F4809180008F7D89
:1038300003C0809180008F7780938000089584B5C5
:103840008F7702C084B58F7D84BD08958091B000CC
:103850008F7703C08091B0008F7D8093B000089572
:10386000CF93DF9390E0FC01E458FF4F2491FC01DB
:10387000E057FF4F8491882349F190E0880F991F0A
:10388000FC01E854FF4FA591B49182559F4FFC0174
:10389000C591D4919FB7611108C0F8948C9120957F
:1038A00082238C93888182230AC0623051F4F89479
:1038B0008C91322F309583238C938881822B88833F
:1038C00004C0F8948C91822B8C939FBFDF91CF9191
:1038D0000895A1E0B0E0EFE6FCE10C94B920282FB8
:1038E00030E0F901E859FF4F8491F901E458FF4FA6
:1038F0001491F901E057FF4F04910023C9F0882388
:1039000021F069830E94071C6981E02FF0E0EE0F2F
:10391000FF1FE255FF4FA591B4919FB7F8948C918A
:10392000611103C01095812301C0812B8C939FBF2F
:103930002196E4E00C94D520CF93DF93282F30E03C
:10394000F901E859FF4F8491F901E458FF4FD491F0
:10395000F901E057FF4FC491CC2391F081110E94EF
:10396000071CEC2FF0E0EE0FFF1FEC55FF4FA59169
:10397000B4912C912D2381E090E021F480E002C0ED
:1039800080E090E0DF91CF9108958E3008F08E5066
:1039900087702091BD0190E4299F90011124822B12
:1039A00080937C0080917A00806480937A0080917B
:1039B0007A0086FDFCCF809178002091790090E01C
:1039C000922B0895A0E0B0E0E8EEFCE10C94B52065
:1039D0006C017A01EB01E60EF71E00E010E0CE1557
:1039E000DF0561F06991D601ED91FC910190F081C4
:1039F000E02DC6010995080F191FF1CFC801CDB7F9
:103A0000DEB7E8E00C94D1206115710589F0DB0187
:103A10000D900020E9F7AD0141505109461B570BAD
:103A2000DC01ED91FC910280F381E02D0995089570
:103A300080E090E008950E94041D0895DC01ED915E
:103A4000FC910190F081E02D099508950F931F934B
:103A5000CF93DF93EC016DE00E941E1D8C016AE0A4
:103A6000CE010E941E1D800F911FDF91CF911F91EB
:103A70000F9108950F931F93CF93DF93EC010E9452
:103A8000041D8C01CE010E94261D800F911FDF9125
:103A9000CF911F910F9108950F931F93CF93DF93B1
:103AA000EC010E941E1D8C01CE010E94261D800F7C
:103AB000911FDF91CF911F910F910895A1E2B0E086
:103AC000E4E6FDE10C94B1207C01C42EE52FCB018E
:103AD000D22E19A221E02D1510F02AE0D22E8E014F
:103AE0000F5D1F4F8D2C912CA12CB12C6C2D7E2F96
:103AF000A50194010E946A208C2DD29E8019112468
:103B0000015011098A3010F4805D01C0895CF80110
:103B10008083211531054105510521F0C22EE32F87
:103B2000CA01E4CFB801C7010E94041DA196ECE0D0
:103B30000C94CD20A0E0B0E0E0EAFDE10C94B520CB
:103B4000EC016A017B012115310541F4E881F9811D
:103B50000190F081E02D642F09951DC02A303105B8
:103B6000A9F477FF12C06DE20E941E1D8C0144274C
:103B70005527BA014C195D096E097F092AE0CE016B
:103B80000E945E1D800F911F06C02AE0B701A601AA
:103B9000CE010E945E1DCDB7DEB7E8E00C94D120C7
:103BA0000F931F93CF93DF93EC019A01AB0166272C
:103BB00057FD6095762F0E949A1D8C01CE010E94C0
:103BC000261D800F911FDF91CF911F910F910895B6
:103BD0002115310549F4DC01ED91FC910190F08152
:103BE000E02D642F099508950E945E1D08959A01A5
:103BF000462F50E060E070E00E94E81D08959A01B1
:103C0000AB0160E070E00E94E81D0895FC0124858E
:103C10003585F901E05CFF4F80819181F901EE5B10
:103C2000FF4F20813181821B930B8F739927089559
:103C3000FC0184859585FC01E05CFF4F408151814A
:103C4000FC01EE5BFF4F208131814217530741F0A9
:103C50000190F081E02DE80FF91F808190E0089538
:103C60008FEF9FEF0895FC0184859585FC01E05C52
:103C7000FF4F40815181FC01EE5BFF4F208131817C
:103C80004217530779F0A081B181A80FB91F8C9119
:103C9000208131812F5F3F4F2F7333273183208362
:103CA00090E008958FEF9FEF0895FC0181A1882394
:103CB00029F0A489B5898C9186FFFBCF11A20895C4
:103CC000CF93DF93FC0126853785D901A05CBF4FD8
:103CD0008D919C91119701968F739927E901CE5B85
:103CE000DF4F4881598184179507D9F30D90BC9116
:103CF000A02DA20FB31F6C93A685B785A05CBF4F04
:103D000011969C938E93A689B7892C9181E090E0BF
:103D1000078C02C0880F991F0A94E2F7282B2C9376
:103D200081E081A30488F589E02D8081806480830F
:103D300081E090E0DF91CF91089508951F920F9256
:103D40000FB60F9211242F933F934F938F939F930E
:103D5000EF93FF938091C00082FD1CC04091C6008C
:103D60008091B8049091B90401968F73992720919E
:103D7000BA043091BB048217930771F0E091B80444
:103D8000F091B904E858FB4F40839093B9048093B5
:103D9000B80402C08091C600FF91EF919F918F916E
:103DA0004F913F912F910F900FBE0F901F9018953C
:103DB00082E194E00E94061E892B11F00E949D1E54
:103DC00008951F920F920FB60F9211242F933F93D5
:103DD0008F939F93EF93FF93209174043091750418
:103DE00080917604909177042817390731F48091F7
:103DF000C1008F7D8093C10014C0E0917604F091E2
:103E00007704EC5CFB4F20818091760490917704DD
:103E100001968F739927909377048093760420936B
:103E2000C600FF91EF919F918F913F912F910F903D
:103E30000FBE0F901F901895A0E0B0E0E2E2FFE106
:103E40000C94B120FC011382128288EE93E0A0E072
:103E5000B0E084839583A683B78386EC92E0918358
:103E600080837587648757874687318B208B138BB8
:103E7000028BF58AE48AD78AC68AB18EA08E938E89
:103E8000828E8F85848F8889858F8989868F8A899C
:103E9000878F8B8980A3ECE00C94CD20CF92DF92AA
:103EA000EF92FF92CF93DF93EC016A017B01411502
:103EB00081EE580761057105F9F0EC89FD8981E013
:103EC00090E008A002C0880F991F0A94E2F780834F
:103ED00060E079E08DE390E0A70196010E946A20FE
:103EE0002150310941095109569547953795279534
:103EF000211580E1380798F0EC89FD89108260E88F
:103F000074E88EE190E0A70196010E946A2021509A
:103F10003109410951095695479537952795E88903
:103F2000F9893083EA89FB89208319A2EE89FF8908
:103F3000408181E090E09C010C8C02C0220F331F75
:103F40000A94E2F7422B4083EE89FF8940819C016D
:103F50000D8C02C0220F331F0A94E2F7422B4083DC
:103F6000EE89FF8940819C010E8C02C0220F331F15
:103F70000A94E2F7422B4083EE89FF8920810F8C5F
:103F800002C0880F991F0A94E2F7809582238083EC
:103F9000DF91CF91FF90EF90DF90CF9008958F92B7
:103FA0009F92AF92BF92CF92DF92EF92FF920F93C8
:103FB0001F9381E08F9385E08F9387E08F9383E059
:103FC0008F9384E08F93E6EC8E2E912CF2ECAF2E43
:103FD000B12CA1ECCA2ED12CB0ECEB2EF12C04ECC0
:103FE00010E025EC30E044E354E068E774E082E15F
:103FF00094E00E941C1F0F900F900F900F900F9055
:104000001F910F91FF90EF90DF90CF90BF90AF90F6
:104010009F908F9008950E94CC1B0E945C12C8ED67
:10402000DEE10E9452162097E1F30E94D81EF9CFDC
:10403000A29FB001B39FC001A39F700D811D1124E9
:10404000911DB29F700D811D1124911D08950E9434
:104050001820A59F900DB49F900DA49F800D911DD9
:1040600011240895B7FF0C9427200E942720821B5B
:10407000930B0895DB018F939F930E942720BF919C
:10408000AF91A29F800D911DA39F900DB29F900DA7
:1040900011240895991B79E004C0991F961708F020
:1040A000961B881F7A95C9F780950895AA1BBB1B9C
:1040B00051E107C0AA1FBB1FA617B70710F0A61B28
:1040C000B70B881F991F5A95A9F780959095BC0149
:1040D000CD010895A1E21A2EAA1BBB1BFD010DC044
:1040E000AA1FBB1FEE1FFF1FA217B307E407F507A8
:1040F00020F0A21BB30BE40BF50B661F771F881F84
:10410000991F1A9469F760957095809590959B0119
:10411000AC01BD01CF010895052E97FB1EF400945C
:104120000E94A32057FD07D00E946A2007FC03D0FD
:104130004EF40C94A32050954095309521953F4F17
:104140004F4F5F4F089590958095709561957F4F83
:104150008F4F9F4F08952F923F924F925F926F9291
:104160007F928F929F92AF92BF92CF92DF92EF9207
:10417000FF920F931F93CF93DF93CDB7DEB7CA1B88
:10418000DB0B0FB6F894DEBF0FBECDBF09942A88B3
:10419000398848885F846E847D848C849B84AA845B
:1041A000B984C884DF80EE80FD800C811B81AA81E8
:1041B000B981CE0FD11D0FB6F894DEBF0FBECDBFB3
:1041C000ED010895EE0FFF1F0590F491E02D099485
:1041D000FB01DC0102C001900D9241505040D8F724
:1041E0000895F999FECF92BD81BDF89A992780B5BF
:1041F0000895262FF999FECF1FBA92BD81BD20BD2B
:104200000FB6F894FA9AF99A0FBE01960895F894A9
:02421000FFCFDE
:104212000000BC04200008409CFF0088130002003C
:10422200020002000200020002000200020002007C
:10423200020002000200020002000200020020014D
:10424200220126022102270323032604260526052E
:104252002B0624072507280729072A8025000005A1
:10426200400AA1204EA50020244EA52C2330C012C6
:1042720000001A400AA1204EA5001B1E27522C2323
:10428200308025000005400AA1204EA50020244EC2
:10429200A52C2330004B000006400AD0009D4900A7
:1042A2007B289D492C233000E1000005400A45018E
:1042B200D7DC03B81E0EBF00232E48E801008A4057
:1042C2000A6001555502AD1E20000023C801545852
:1042D2002074696D656F7574210057616974696E28
:1042E200672062696E640A00476F7420706B740AFB
:1042F200006461746120676F6F640A007363616EAA
:104302006E6572206D6F6465004F70656E4C52531E
:104312006E67205258207374617274696E67200050
:10432200206F6E20485720005361766564206269D1
:104332006E64206461746120746F20454550524F51
:104342004D0A004920616D20736C61766500456EEF
:10435200746572696E67206E6F726D616C206D6F2D
:10436200646500454550524F4D2064617461206E72
:104372006F742076616C6964206F722062696E646A
:10438200206A756D70706572207365742C20666F7B
:104392007263696E672062696E640A00525820680F
:1043A200616E6700B200F4014C0300070B0C1011A0
:1043B2001500091203130E0F000102000000100085
:1043C20000000800200000010000020000000100BF
:1043D200000200000000601EE21C061E331E181EB2
:0243E200551E66
:107E00000F92CDB7DEB7112484B714BE81FFF1D035
:107E100082E08093C00088E18093C10086E0809377
:107E2000C20080E18093C4008EE0CDD088249924E4
:107E3000CC24C394F5E0DF2EE1E1EE2E73E0F72EC3
:107E4000B6D0082F813479F4B2D08983C2D0898129
:107E5000823811F481E005C0813811F485E001C059
:107E600083E09ED09AC0823411F484E103C085344B
:107E700019F485E0B6D091C0853561F498D0082F0B
:107E800010E095D090E0982E8824802A912A880CC2
:107E9000991C82C0863521F484E0A3D080E0E1CF34
:107EA000843609F04CC083D082D0A82E80D0B82E62
:107EB00000E011E07CD0F80181938F01AE16D1F77C
:107EC00088D0FB2DF53489F4E0E0F1E00BC0F9999E
:107ED000FECF92BC81BC0894811C911C819180BD15
:107EE000FA9AF99AEA1598F358C08B2D863409F05E
:107EF00054C0F401F7BEE89507B600FCFDCFF401CD
:107F0000A0E0B1E02C9130E011968C91119790E0B7
:107F1000982F8827822B932B12960C01C7BEE895C9
:107F20001124329681E0A038B80761F7F401D7BE7A
:107F3000E89507B600FCFDCFE7BEE8952EC0843774
:107F4000F1F435D034D0182F32D0B82E42D0FB2DDA
:107F5000F63421F4F40105914F010CC0FB2DF534EA
:107F600049F4F999FECF92BC81BC0894811C911C04
:107F7000F89A00B5802F14D0115049F70EC08537FC
:107F800039F427D08EE10CD085E90AD08FE069CF93
:107F9000813511F488E017D01CD080E101D050CF9A
:107FA0009091C00095FFFCCF8093C600089580910A
:107FB000C00087FFFCCF8091C00084FD01C0A89560
:107FC0008091C6000895E0E6F0E098E19083808318
:107FD0000895EDDF803219F088E0F5DFFFCF84E10E
:107FE000DFCF1F93182FE3DF1150E9F7F2DF1F9166
:0E7FF0000895282E80E0E7DFEE27FF27099492
:027FFE0001057B
:0400000300007E007B
:00000001FF
